BL51 BANKED LINKER/LOCATER V5.01                                                        03/27/2012  17:23:10  PAGE 1


BL51 BANKED LINKER/LOCATER V5.01, INVOKED BY:
C:\KEIL\C51\BIN\BL51.EXE expert2.obj TO expert2


INPUT MODULES INCLUDED:
  expert2.obj (EXPERT2)


LINK MAP OF MODULE:  expert2 (EXPERT2)


            TYPE    BASE      LENGTH    RELOCATION   SEGMENT NAME
            -----------------------------------------------------

            * * * * * * *   D A T A   M E M O R Y   * * * * * * *
            REG     0000H     0008H     ABSOLUTE     "REG BANK 0"

            * * * * * * *   C O D E   M E M O R Y   * * * * * * *
            CODE    0000H     057BH     ABSOLUTE     



SYMBOL TABLE OF MODULE:  expert2 (EXPERT2)

  VALUE           TYPE          NAME
  ----------------------------------

  -------         MODULE        EXPERT2
  B:00A0H.0       SYMBOL        A0_8255
  B:00A0H.1       SYMBOL        A1_8255
  N:0055H         SYMBOL        ABUF
  D:00E0H         SYMBOL        ACC
  C:04D5H         SYMBOL        ADCBIT
  C:0169H         SYMBOL        ADC_SCR1
  C:0172H         SYMBOL        ADC_SCR2
  C:04A9H         SYMBOL        ADC_SUBP
  N:0020H         SYMBOL        ADRS_9346
  C:0120H         SYMBOL        ADVAN_SCR1
  C:012EH         SYMBOL        ADVAN_SCR2
  C:0028H         SYMBOL        ADVLOOP
  N:0054H         SYMBOL        ATMP
  D:00F0H         SYMBOL        B
  C:0348H         SYMBOL        BACK
  N:0057H         SYMBOL        BOUNCE0
  N:0056H         SYMBOL        BOUNCE1
  C:02B0H         SYMBOL        CHECK_KEY
  C:02C7H         SYMBOL        CHKLP
  C:0223H         SYMBOL        CHK_LCDBZY
  C:03F9H         SYMBOL        CLK_PUS
  C:0255H         SYMBOL        CL_PC
  N:0053H         SYMBOL        CNY70
  N:0058H         SYMBOL        COUNTER
  N:0076H         SYMBOL        COUNT_0832
  N:007EH         SYMBOL        COUNT_164
  N:0074H         SYMBOL        COUNT_9346
  N:005FH         SYMBOL        CTRL55
  N:0073H         SYMBOL        DATA_HB
  N:0072H         SYMBOL        DATA_LB
BL51 BANKED LINKER/LOCATER V5.01                                                      03/27/2012  17:23:10  PAGE 2


  C:03CFH         SYMBOL        DATA_PRO
  C:02C1H         SYMBOL        DBLCHK
  C:032AH         SYMBOL        DCMNT2
  C:032FH         SYMBOL        DCMNT3
  C:0334H         SYMBOL        DCMNT4
  C:0339H         SYMBOL        DCMOVER
  C:014AH         SYMBOL        DCM_B
  C:0148H         SYMBOL        DCM_F
  C:014CH         SYMBOL        DCM_L
  C:014EH         SYMBOL        DCM_R
  C:013FH         SYMBOL        DCM_SCR1
  C:0147H         SYMBOL        DCM_SCR2
  C:0325H         SYMBOL        DCM_SUBP
  C:037BH         SYMBOL        DL1
  C:037EH         SYMBOL        DL2
  C:0198H         SYMBOL        ENDPS
  C:045DH         SYMBOL        ERASEWAIT
  C:044BH         SYMBOL        ERASE_DATA
  C:043FH         SYMBOL        EW_DIS
  C:0433H         SYMBOL        EW_ENA
  C:033AH         SYMBOL        FORWARD
  C:0051H         SYMBOL        FUNCT1
  C:005BH         SYMBOL        FUNCT11
  C:006CH         SYMBOL        FUNCT12
  C:0075H         SYMBOL        FUNCT2
  C:007FH         SYMBOL        FUNCT21
  C:00ABH         SYMBOL        FUNCT3
  C:00EFH         SYMBOL        FUNCT31
  C:02EDH         SYMBOL        GREEN
  C:02A9H         SYMBOL        HAVE_STATE
  C:0000H         SYMBOL        INITIAL
  C:02AFH         SYMBOL        IS_KEY
  C:0039H         SYMBOL        JUDGEKEY
  N:0059H         SYMBOL        KEYDBL
  N:005AH         SYMBOL        KEYNUM
  B:0022H.0       SYMBOL        KEY_F
  C:0173H         SYMBOL        LCD_CLS
  C:0179H         SYMBOL        LCD_HOME
  C:017FH         SYMBOL        LCD_LOCATE
  C:018DH         SYMBOL        LCD_PRINTSTRING
  C:0199H         SYMBOL        LCD_RDPOST
  B:0022H.1       SYMBOL        LED_FLG
  B:00A0H.3       SYMBOL        LED_GRN
  B:00A0H.2       SYMBOL        LED_RED
  C:0356H         SYMBOL        LEFT
  C:0311H         SYMBOL        LOOP_164
  C:010EH         SYMBOL        MAIN_SCR1
  C:0116H         SYMBOL        MAIN_SCR2
  C:015FH         SYMBOL        MEM_CODE
  C:03EBH         SYMBOL        MEM_RD
  C:0156H         SYMBOL        MEM_SCR1
  C:015EH         SYMBOL        MEM_SCR2
  C:03DDH         SYMBOL        MEM_WR
  B:00A0H.6       SYMBOL        ML1
  B:00A0H.7       SYMBOL        ML2
  B:00A0H.4       SYMBOL        MR1
  B:00A0H.5       SYMBOL        MR2
BL51 BANKED LINKER/LOCATER V5.01                                                      03/27/2012  17:23:10  PAGE 3


  N:006FH         SYMBOL        MTR_CNT0
  N:006EH         SYMBOL        MTR_CNT1
  N:006DH         SYMBOL        MTR_TIME
  C:0300H         SYMBOL        NEXT164
  C:0042H         SYMBOL        NEXTJ1
  C:0047H         SYMBOL        NEXTJ2
  C:004CH         SYMBOL        NEXTJ3
  C:009BH         SYMBOL        NEXTJG
  C:02B8H         SYMBOL        NEXTK
  C:0088H         SYMBOL        NEXTSN
  C:01A8H         SYMBOL        NOTSEC
  C:02DDH         SYMBOL        NOT_KEY
  C:02F2H         SYMBOL        NUMBER_SET
  C:031BH         SYMBOL        NUMCODE
  C:0150H         SYMBOL        OPS_SCR1
  C:0155H         SYMBOL        OPS_SCR2
  C:038BH         SYMBOL        OPS_SUBP
  C:030DH         SYMBOL        OUT_H
  D:0090H         SYMBOL        P1
  D:00A0H         SYMBOL        P2
  D:00B0H         SYMBOL        P3
  N:005EH         SYMBOL        PA55
  N:005DH         SYMBOL        PB55
  N:005CH         SYMBOL        PC55
  N:005BH         SYMBOL        PCBIT
  C:0422H         SYMBOL        RDBIT
  C:042BH         SYMBOL        RDH
  C:042DH         SYMBOL        RDLP9346
  C:041EH         SYMBOL        RD_BYTE
  C:01F5H         SYMBOL        RD_LCDCOM
  C:023BH         SYMBOL        RD_PA
  C:0243H         SYMBOL        RD_PB
  C:04D1H         SYMBOL        READ_ADC
  C:048EH         SYMBOL        READ_DATA
  C:02E8H         SYMBOL        RED
  C:0364H         SYMBOL        RIGHT
  C:037BH         SYMBOL        RUN_DL
  B:00B0H.0       SYMBOL        S0832_CLK
  B:00B0H.1       SYMBOL        S0832_CS
  B:00B0H.3       SYMBOL        S0832_DI
  B:00B0H.4       SYMBOL        S0832_DO
  C:0315H         SYMBOL        S164CLK
  B:0090H.7       SYMBOL        S74CLK
  B:0090H.6       SYMBOL        S74CLR
  B:0090H.0       SYMBOL        S74DTA
  B:0090H.1       SYMBOL        S9346_CLK
  B:0090H.0       SYMBOL        S9346_CS
  B:0090H.2       SYMBOL        S9346_DI
  B:0090H.3       SYMBOL        S9346_DO
  C:025FH         SYMBOL        SCAN_KEY
  C:0186H         SYMBOL        SETB7
  C:00D6H         SYMBOL        SHOW_DT
  C:008FH         SYMBOL        SHO_0
  C:0096H         SYMBOL        SHO_1
  C:002FH         SYMBOL        SHO_ADVAN
  C:0101H         SYMBOL        SHO_LCM1
  C:0106H         SYMBOL        SHO_LCM2
BL51 BANKED LINKER/LOCATER V5.01                                                      03/27/2012  17:23:10  PAGE 4


  C:001EH         SYMBOL        SHO_MAIN
  C:0372H         SYMBOL        STOP
  C:024BH         SYMBOL        ST_PC
  N:0052H         SYMBOL        TDL70
  C:02E3H         SYMBOL        TEAM_SET
  N:0077H         SYMBOL        TEMP_0832
  N:007FH         SYMBOL        TEMP_164
  N:0075H         SYMBOL        TEMP_9346
  C:0409H         SYMBOL        WRBIT
  C:0416H         SYMBOL        WRH
  C:0464H         SYMBOL        WRITE_DATA
  C:041AH         SYMBOL        WRLP9346
  C:0485H         SYMBOL        WRWAIT
  C:0406H         SYMBOL        WR_BYTE
  C:022BH         SYMBOL        WR_CTRL
  C:01CFH         SYMBOL        WR_LCDCMD
  C:01A9H         SYMBOL        WR_LCDDAT
  C:04B6H         SYMBOL        WR_OPCODE
  C:0233H         SYMBOL        WR_PA
  C:03FFH         SYMBOL        WR_SB
  C:03D6H         SYMBOL        Y70_DL
  C:0000H         LINE#         76
  C:0003H         LINE#         77
  C:0005H         LINE#         80
  C:0008H         LINE#         81
  C:000AH         LINE#         83
  C:000DH         LINE#         84
  C:000FH         LINE#         86
  C:0012H         LINE#         87
  C:0014H         LINE#         89
  C:0016H         LINE#         90
  C:0018H         LINE#         92
  C:001AH         LINE#         93
  C:001CH         LINE#         95
  C:001EH         LINE#         98
  C:0021H         LINE#         99
  C:0023H         LINE#         100
  C:0026H         LINE#         101
  C:0028H         LINE#         104
  C:002AH         LINE#         105
  C:002CH         LINE#         106
  C:002FH         LINE#         109
  C:0032H         LINE#         110
  C:0034H         LINE#         111
  C:0037H         LINE#         112
  C:0039H         LINE#         114
  C:003BH         LINE#         115
  C:003DH         LINE#         116
  C:0040H         LINE#         117
  C:0042H         LINE#         118
  C:0045H         LINE#         119
  C:0047H         LINE#         120
  C:004AH         LINE#         121
  C:004CH         LINE#         122
  C:004FH         LINE#         123
  C:0051H         LINE#         126
  C:0054H         LINE#         127
BL51 BANKED LINKER/LOCATER V5.01                                                      03/27/2012  17:23:10  PAGE 5


  C:0056H         LINE#         128
  C:0059H         LINE#         129
  C:005BH         LINE#         131
  C:005DH         LINE#         132
  C:005FH         LINE#         133
  C:0061H         LINE#         134
  C:0062H         LINE#         135
  C:0064H         LINE#         136
  C:0066H         LINE#         137
  C:0068H         LINE#         138
  C:006AH         LINE#         139
  C:006CH         LINE#         141
  C:006EH         LINE#         142
  C:0071H         LINE#         143
  C:0073H         LINE#         144
  C:0075H         LINE#         147
  C:0078H         LINE#         148
  C:007AH         LINE#         149
  C:007DH         LINE#         150
  C:007FH         LINE#         152
  C:0081H         LINE#         153
  C:0083H         LINE#         154
  C:0084H         LINE#         155
  C:0086H         LINE#         156
  C:0088H         LINE#         157
  C:008AH         LINE#         158
  C:008BH         LINE#         159
  C:008DH         LINE#         160
  C:008FH         LINE#         161
  C:0092H         LINE#         162
  C:0094H         LINE#         163
  C:0096H         LINE#         164
  C:0099H         LINE#         165
  C:009BH         LINE#         166
  C:009DH         LINE#         168
  C:00A0H         LINE#         169
  C:00A2H         LINE#         171
  C:00A4H         LINE#         172
  C:00A6H         LINE#         173
  C:00A9H         LINE#         174
  C:00ABH         LINE#         177
  C:00AEH         LINE#         178
  C:00B0H         LINE#         179
  C:00B3H         LINE#         180
  C:00B5H         LINE#         182
  C:00B7H         LINE#         183
  C:00B9H         LINE#         184
  C:00BCH         LINE#         185
  C:00BDH         LINE#         186
  C:00BEH         LINE#         188
  C:00C0H         LINE#         189
  C:00C3H         LINE#         190
  C:00C4H         LINE#         191
  C:00C5H         LINE#         193
  C:00C7H         LINE#         194
  C:00CAH         LINE#         195
  C:00CBH         LINE#         196
BL51 BANKED LINKER/LOCATER V5.01                                                      03/27/2012  17:23:10  PAGE 6


  C:00CEH         LINE#         197
  C:00CFH         LINE#         198
  C:00D0H         LINE#         200
  C:00D1H         LINE#         201
  C:00D3H         LINE#         202
  C:00D5H         LINE#         203
  C:00D6H         LINE#         205
  C:00D9H         LINE#         206
  C:00DAH         LINE#         207
  C:00DBH         LINE#         208
  C:00DDH         LINE#         209
  C:00DFH         LINE#         210
  C:00E2H         LINE#         211
  C:00E4H         LINE#         212
  C:00E5H         LINE#         213
  C:00E6H         LINE#         214
  C:00E8H         LINE#         215
  C:00EAH         LINE#         216
  C:00EDH         LINE#         217
  C:00EFH         LINE#         219
  C:00F1H         LINE#         220
  C:00F3H         LINE#         221
  C:00F5H         LINE#         222
  C:00F6H         LINE#         223
  C:00F8H         LINE#         225
  C:00FAH         LINE#         226
  C:00FCH         LINE#         227
  C:00FFH         LINE#         228
  C:0101H         LINE#         232
  C:0103H         LINE#         233
  C:0105H         LINE#         234
  C:0106H         LINE#         236
  C:0107H         LINE#         237
  C:0109H         LINE#         238
  C:010BH         LINE#         239
  C:010DH         LINE#         240
  C:0173H         LINE#         266
  C:0176H         LINE#         267
  C:0178H         LINE#         268
  C:0179H         LINE#         271
  C:017CH         LINE#         272
  C:017EH         LINE#         273
  C:017FH         LINE#         276
  C:0181H         LINE#         277
  C:0184H         LINE#         278
  C:0186H         LINE#         279
  C:0188H         LINE#         280
  C:018AH         LINE#         281
  C:018CH         LINE#         282
  C:018DH         LINE#         285
  C:018EH         LINE#         286
  C:018FH         LINE#         287
  C:0191H         LINE#         288
  C:0193H         LINE#         289
  C:0195H         LINE#         290
  C:0196H         LINE#         291
  C:0198H         LINE#         292
BL51 BANKED LINKER/LOCATER V5.01                                                      03/27/2012  17:23:10  PAGE 7


  C:0199H         LINE#         295
  C:019BH         LINE#         296
  C:019DH         LINE#         297
  C:019FH         LINE#         298
  C:01A1H         LINE#         299
  C:01A4H         LINE#         300
  C:01A6H         LINE#         301
  C:01A8H         LINE#         302
  C:01A9H         LINE#         305
  C:01ABH         LINE#         306
  C:01AEH         LINE#         307
  C:01B0H         LINE#         308
  C:01B3H         LINE#         309
  C:01B5H         LINE#         310
  C:01B8H         LINE#         311
  C:01BAH         LINE#         312
  C:01BDH         LINE#         313
  C:01BFH         LINE#         314
  C:01C2H         LINE#         315
  C:01C4H         LINE#         316
  C:01C7H         LINE#         317
  C:01C9H         LINE#         318
  C:01CCH         LINE#         319
  C:01CEH         LINE#         320
  C:01CFH         LINE#         323
  C:01D1H         LINE#         324
  C:01D4H         LINE#         325
  C:01D6H         LINE#         326
  C:01D9H         LINE#         327
  C:01DBH         LINE#         328
  C:01DEH         LINE#         329
  C:01E0H         LINE#         330
  C:01E3H         LINE#         331
  C:01E5H         LINE#         332
  C:01E8H         LINE#         333
  C:01EAH         LINE#         334
  C:01EDH         LINE#         335
  C:01EFH         LINE#         336
  C:01F2H         LINE#         337
  C:01F4H         LINE#         338
  C:01F5H         LINE#         341
  C:01F8H         LINE#         342
  C:01FAH         LINE#         344
  C:01FDH         LINE#         345
  C:01FFH         LINE#         346
  C:0202H         LINE#         347
  C:0204H         LINE#         348
  C:0207H         LINE#         349
  C:0209H         LINE#         350
  C:020BH         LINE#         351
  C:020EH         LINE#         352
  C:0211H         LINE#         353
  C:0213H         LINE#         354
  C:0216H         LINE#         355
  C:0218H         LINE#         356
  C:021BH         LINE#         357
  C:021DH         LINE#         359
BL51 BANKED LINKER/LOCATER V5.01                                                      03/27/2012  17:23:10  PAGE 8


  C:0220H         LINE#         360
  C:0222H         LINE#         361
  C:0223H         LINE#         364
  C:0225H         LINE#         365
  C:0227H         LINE#         366
  C:022AH         LINE#         367
  C:022BH         LINE#         371
  C:022DH         LINE#         372
  C:022FH         LINE#         373
  C:0231H         LINE#         374
  C:0232H         LINE#         375
  C:0233H         LINE#         378
  C:0235H         LINE#         379
  C:0237H         LINE#         380
  C:0239H         LINE#         381
  C:023AH         LINE#         382
  C:023BH         LINE#         385
  C:023DH         LINE#         386
  C:023FH         LINE#         387
  C:0240H         LINE#         388
  C:0242H         LINE#         389
  C:0243H         LINE#         392
  C:0245H         LINE#         393
  C:0247H         LINE#         394
  C:0248H         LINE#         395
  C:024AH         LINE#         396
  C:024BH         LINE#         399
  C:024DH         LINE#         400
  C:024FH         LINE#         401
  C:0251H         LINE#         402
  C:0252H         LINE#         403
  C:0253H         LINE#         404
  C:0254H         LINE#         405
  C:0255H         LINE#         408
  C:0257H         LINE#         409
  C:0259H         LINE#         410
  C:025BH         LINE#         411
  C:025CH         LINE#         412
  C:025DH         LINE#         413
  C:025EH         LINE#         414
  C:025FH         LINE#         417
  C:0262H         LINE#         418
  C:0264H         LINE#         421
  C:0267H         LINE#         422
  C:0269H         LINE#         423
  C:026CH         LINE#         424
  C:026EH         LINE#         425
  C:0270H         LINE#         426
  C:0272H         LINE#         427
  C:0275H         LINE#         429
  C:0278H         LINE#         430
  C:027AH         LINE#         431
  C:027DH         LINE#         432
  C:027FH         LINE#         433
  C:0281H         LINE#         434
  C:0283H         LINE#         435
  C:0286H         LINE#         437
BL51 BANKED LINKER/LOCATER V5.01                                                      03/27/2012  17:23:10  PAGE 9


  C:0289H         LINE#         438
  C:028BH         LINE#         439
  C:028EH         LINE#         440
  C:0290H         LINE#         441
  C:0292H         LINE#         442
  C:0294H         LINE#         443
  C:0297H         LINE#         445
  C:029AH         LINE#         446
  C:029CH         LINE#         447
  C:029FH         LINE#         448
  C:02A1H         LINE#         449
  C:02A3H         LINE#         450
  C:02A5H         LINE#         451
  C:02A8H         LINE#         453
  C:02A9H         LINE#         456
  C:02ABH         LINE#         457
  C:02AEH         LINE#         458
  C:02AFH         LINE#         461
  C:02B0H         LINE#         464
  C:02B3H         LINE#         465
  C:02B5H         LINE#         466
  C:02B8H         LINE#         467
  C:02B9H         LINE#         468
  C:02BBH         LINE#         469
  C:02BDH         LINE#         470
  C:02C0H         LINE#         471
  C:02C1H         LINE#         473
  C:02C4H         LINE#         474
  C:02C7H         LINE#         475
  C:02CAH         LINE#         476
  C:02CDH         LINE#         477
  C:02D0H         LINE#         478
  C:02D2H         LINE#         479
  C:02D5H         LINE#         480
  C:02D7H         LINE#         481
  C:02DAH         LINE#         482
  C:02DCH         LINE#         483
  C:02DDH         LINE#         484
  C:02DFH         LINE#         485
  C:02E2H         LINE#         486
  C:02E3H         LINE#         489
  C:02E6H         LINE#         490
  C:02E8H         LINE#         493
  C:02EAH         LINE#         494
  C:02ECH         LINE#         495
  C:02EDH         LINE#         498
  C:02EFH         LINE#         499
  C:02F1H         LINE#         500
  C:02F2H         LINE#         503
  C:02F5H         LINE#         504
  C:02F6H         LINE#         505
  C:02F8H         LINE#         506
  C:02FBH         LINE#         507
  C:02FDH         LINE#         508
  C:02FEH         LINE#         509
  C:0300H         LINE#         512
  C:0302H         LINE#         513
BL51 BANKED LINKER/LOCATER V5.01                                                      03/27/2012  17:23:10  PAGE 10


  C:0303H         LINE#         514
  C:0305H         LINE#         516
  C:0307H         LINE#         517
  C:0309H         LINE#         518
  C:030BH         LINE#         519
  C:030DH         LINE#         520
  C:030FH         LINE#         521
  C:0311H         LINE#         524
  C:0314H         LINE#         525
  C:0315H         LINE#         528
  C:0317H         LINE#         529
  C:0318H         LINE#         530
  C:031AH         LINE#         531
  C:0325H         LINE#         538
  C:0328H         LINE#         539
  C:032AH         LINE#         540
  C:032DH         LINE#         541
  C:032FH         LINE#         542
  C:0332H         LINE#         543
  C:0334H         LINE#         544
  C:0337H         LINE#         545
  C:0339H         LINE#         547
  C:033AH         LINE#         550
  C:033DH         LINE#         551
  C:033FH         LINE#         552
  C:0341H         LINE#         553
  C:0343H         LINE#         554
  C:0345H         LINE#         555
  C:0347H         LINE#         556
  C:0348H         LINE#         559
  C:034BH         LINE#         560
  C:034DH         LINE#         561
  C:034FH         LINE#         562
  C:0351H         LINE#         563
  C:0353H         LINE#         564
  C:0355H         LINE#         565
  C:0356H         LINE#         568
  C:0359H         LINE#         569
  C:035BH         LINE#         570
  C:035DH         LINE#         571
  C:035FH         LINE#         572
  C:0361H         LINE#         573
  C:0363H         LINE#         574
  C:0364H         LINE#         577
  C:0367H         LINE#         578
  C:0369H         LINE#         579
  C:036BH         LINE#         580
  C:036DH         LINE#         581
  C:036FH         LINE#         582
  C:0371H         LINE#         583
  C:0372H         LINE#         586
  C:0374H         LINE#         587
  C:0376H         LINE#         588
  C:0378H         LINE#         589
  C:037AH         LINE#         590
  C:037BH         LINE#         593
  C:037EH         LINE#         594
BL51 BANKED LINKER/LOCATER V5.01                                                      03/27/2012  17:23:10  PAGE 11


  C:0381H         LINE#         595
  C:0384H         LINE#         596
  C:0387H         LINE#         597
  C:038AH         LINE#         598
  C:038BH         LINE#         600
  C:038EH         LINE#         602
  C:0391H         LINE#         603
  C:0393H         LINE#         604
  C:0396H         LINE#         605
  C:0398H         LINE#         606
  C:039AH         LINE#         607
  C:039CH         LINE#         608
  C:039EH         LINE#         610
  C:03A1H         LINE#         611
  C:03A3H         LINE#         612
  C:03A6H         LINE#         613
  C:03A8H         LINE#         614
  C:03AAH         LINE#         615
  C:03ACH         LINE#         616
  C:03AEH         LINE#         618
  C:03B1H         LINE#         619
  C:03B3H         LINE#         620
  C:03B6H         LINE#         621
  C:03B8H         LINE#         622
  C:03BAH         LINE#         623
  C:03BCH         LINE#         624
  C:03BEH         LINE#         626
  C:03C1H         LINE#         627
  C:03C3H         LINE#         628
  C:03C6H         LINE#         629
  C:03C8H         LINE#         630
  C:03CAH         LINE#         631
  C:03CCH         LINE#         632
  C:03CEH         LINE#         634
  C:03CFH         LINE#         637
  C:03D2H         LINE#         638
  C:03D5H         LINE#         639
  C:03D6H         LINE#         642
  C:03D9H         LINE#         643
  C:03DCH         LINE#         644
  C:03DDH         LINE#         648
  C:03DFH         LINE#         649
  C:03E1H         LINE#         650
  C:03E3H         LINE#         651
  C:03E5H         LINE#         653
  C:03E8H         LINE#         654
  C:03EAH         LINE#         655
  C:03EBH         LINE#         658
  C:03EDH         LINE#         659
  C:03EFH         LINE#         660
  C:03F1H         LINE#         661
  C:03F3H         LINE#         663
  C:03F6H         LINE#         664
  C:03F8H         LINE#         665
  C:03F9H         LINE#         669
  C:03FBH         LINE#         670
  C:03FCH         LINE#         671
BL51 BANKED LINKER/LOCATER V5.01                                                      03/27/2012  17:23:10  PAGE 12


  C:03FEH         LINE#         672
  C:03FFH         LINE#         675
  C:0401H         LINE#         676
  C:0403H         LINE#         677
  C:0405H         LINE#         678
  C:0406H         LINE#         681
  C:0409H         LINE#         682
  C:040BH         LINE#         683
  C:040CH         LINE#         684
  C:040EH         LINE#         685
  C:0410H         LINE#         686
  C:0412H         LINE#         687
  C:0414H         LINE#         688
  C:0416H         LINE#         689
  C:0418H         LINE#         690
  C:041AH         LINE#         691
  C:041DH         LINE#         692
  C:041EH         LINE#         695
  C:0421H         LINE#         696
  C:0422H         LINE#         697
  C:0424H         LINE#         698
  C:0427H         LINE#         699
  C:0428H         LINE#         700
  C:0429H         LINE#         701
  C:042BH         LINE#         702
  C:042CH         LINE#         703
  C:042DH         LINE#         704
  C:0430H         LINE#         705
  C:0432H         LINE#         706
  C:0433H         LINE#         709
  C:0436H         LINE#         710
  C:0438H         LINE#         711
  C:043AH         LINE#         712
  C:043CH         LINE#         713
  C:043EH         LINE#         714
  C:043FH         LINE#         717
  C:0442H         LINE#         718
  C:0444H         LINE#         719
  C:0446H         LINE#         720
  C:0448H         LINE#         721
  C:044AH         LINE#         722
  C:044BH         LINE#         725
  C:044DH         LINE#         726
  C:044FH         LINE#         727
  C:0452H         LINE#         728
  C:0454H         LINE#         729
  C:0456H         LINE#         730
  C:0458H         LINE#         731
  C:045AH         LINE#         732
  C:045BH         LINE#         733
  C:045DH         LINE#         734
  C:045EH         LINE#         735
  C:0461H         LINE#         736
  C:0463H         LINE#         737
  C:0464H         LINE#         741
  C:0466H         LINE#         742
  C:0468H         LINE#         743
BL51 BANKED LINKER/LOCATER V5.01                                                      03/27/2012  17:23:10  PAGE 13


  C:046AH         LINE#         744
  C:046CH         LINE#         745
  C:046FH         LINE#         746
  C:0471H         LINE#         747
  C:0473H         LINE#         748
  C:0474H         LINE#         749
  C:0477H         LINE#         750
  C:0479H         LINE#         751
  C:047CH         LINE#         752
  C:047EH         LINE#         753
  C:0480H         LINE#         754
  C:0482H         LINE#         755
  C:0483H         LINE#         756
  C:0485H         LINE#         757
  C:0486H         LINE#         758
  C:0489H         LINE#         759
  C:048BH         LINE#         760
  C:048DH         LINE#         761
  C:048EH         LINE#         764
  C:0490H         LINE#         765
  C:0492H         LINE#         766
  C:0495H         LINE#         767
  C:0497H         LINE#         768
  C:0499H         LINE#         769
  C:049AH         LINE#         770
  C:049CH         LINE#         771
  C:049FH         LINE#         772
  C:04A1H         LINE#         773
  C:04A4H         LINE#         774
  C:04A6H         LINE#         775
  C:04A8H         LINE#         776
  C:04A9H         LINE#         779
  C:04ABH         LINE#         780
  C:04ADH         LINE#         781
  C:04AFH         LINE#         782
  C:04B1H         LINE#         784
  C:04B3H         LINE#         785
  C:04B5H         LINE#         786
  C:04B6H         LINE#         790
  C:04B8H         LINE#         791
  C:04BAH         LINE#         792
  C:04BCH         LINE#         793
  C:04BEH         LINE#         794
  C:04C0H         LINE#         796
  C:04C2H         LINE#         797
  C:04C4H         LINE#         798
  C:04C6H         LINE#         799
  C:04C8H         LINE#         801
  C:04CAH         LINE#         802
  C:04CCH         LINE#         803
  C:04CEH         LINE#         804
  C:04D0H         LINE#         805
  C:04D1H         LINE#         808
  C:04D4H         LINE#         809
  C:04D5H         LINE#         810
  C:04D7H         LINE#         811
  C:04D9H         LINE#         812
BL51 BANKED LINKER/LOCATER V5.01                                                      03/27/2012  17:23:10  PAGE 14


  C:04DBH         LINE#         813
  C:04DCH         LINE#         814
  C:04DFH         LINE#         815
  C:04E1H         LINE#         816
  C:04E3H         LINE#         817
  -------         ENDMOD        EXPERT2

******************************************************************************
* RESTRICTED VERSION WITH 0800H BYTE CODE SIZE LIMIT; USED: 04E8H BYTE (61%) *
******************************************************************************

Program Size: data=8.0 xdata=0 code=1403
LINK/LOCATE RUN COMPLETE.  0 WARNING(S),  0 ERROR(S)
